S123D0007ED0EB7ED1CA7ED34E4D43465320322E302E310D0A002023200008200800457282
S123D020726F723A20004E6F7420666F756E6400416C7265616479206578697374004E6F06
S123D040207370616365206C656674004E6F7420656D707479004D697373696E67206F727A
S123D060206D616C666F726D656420617267756D656E74004163636573732064656E6965DB
S123D08064004E6F742065786563757461626C6500536176696E6720004C6F6164696E676F
S123D0A0200053797374656D2074696D65206973206E6F74207365740D0A00436F6D6D611B
S123D0C06E64733A0D0A00466F726D61742059595959204D4D204444204848204D4D20538A
S123D0E0530D0A0073797374656D00BDD74186F09702CEBC006F00088CBCEA23F8CED00944
S123D100BDD736BDE1CEBDE1F327037ED116BDE06E26037ED1E4B7BCE6CED01EBDD736CEA1
S123D120BCE6BDD761BDD7417EC0008647BBBC00BBBC01BBBC04BBBC05BBBC06BBBC07BBD8
S123D140BC08BBBC09BBBC0ABBBC0BBBBC0CBBBC0DBBBC0EBBBC0FBBBC10BBBC11BBBC12DA
S123D160BBBC1339B7BCE6CED01EBDD736CEBCE6BDD761BDD7417ED1E416CED02620241668
S123D180CED030201E16CED056201816CED03E201216CED04C200C16CED074200616CED0EB
S123D1A08220003CCED01EBDD73638BDD736BDD74B8628BD7FE8F7BCE6CEBCE6BDD76186D0
S123D1C029BD7FE8BDD7417ED1E486F09702BDD12BB1BCEB27037ED0EBBDE1CEBDE1F3274F
S123D1E0037ED0EBBDE333CEBC14BDD736CED016BDD736CEBCA06F00BD7FEB81082719812C
S123D2000D2727811F23F1817F22ED8CBCDF27E8BD7FE8A7000820E08CBCA027DB096F0081
S123D2203CCED01ABDD7363820CEBDD7416F008CBCA027B0FEBC10FFBC94FEBC12FFBC96CD
S123D2407ED2D1D262D267D26DD272D27AD281D288D28ED297D2A0D2A7D2AFD2B6D2C0D29F
S123D260CA006C7300D7D864697200D7D8636400D86B6D6B64697200D8FF7361766500D9E4
S123D280B26C6F616400DAD172756E00DB7664656C65746500DB9F72656E616D6500DC0D99
S123D2A06174747200DC96746F75636800DD0674696D6500DD4C73657474696D6500DDA3E4
S123D2C06D6F6E69746F7200DEA168656C7000DEAACED243FFBCE7CEBCA0FFBCE0FEBCE7A7
S123D2E06D0026037ED308EE00BDD71E270AFEBCE70808FFBCE720DF3CCEBCA0FFBCE038DF
S123D30008EE006E007ED1E4FEBC0CFFBC94FEBC0EFFBC96CED0E4FFBCE0BDDFF72702204B
S123D3202AA60084C181C127022020EC01FDBC94EC03FDBC96CEBCA0FFBCE0BDDFF7270230
S123D3402009CCBCA0FDBCE07EE1217ED17986F0970286FFA701BDE1CEBDE1F3270139BD40
S123D360D12BB1BCEB270139FFBCE4FCBC10FDBC94FCBC12FDBC96A600810126037ED3A8DD
S123D380810726037ED403810826037ED469811026037ED4C8811126037ED5428120260328
S123D3A07ED5AC86FEA70139EC02FDBCE0EE02EE008C2E002615FEBCE486C1A704FCBC1251
S123D3C0B3BC10C30001ED056F0139BDDFF7262DFFBCE7A600FEBCE4A704FEBCE7EC03A3C1
S123D3E001C30001FEBCE4ED05C605FEBCE73AA600FEBCE43AA7025CC10F23EF4FFEBCE4DC
S123D400A70139EE04FFBCE0BDD77025037ED465BDDFF726037ED465FEBCE4EE02FFBCE01B
S123D420BDDFF727037ED465A600850226037ED4653CFEBCE4EE04FFBCE038C6103AC61FD3
S123D440BDD67B4D270A81202706A700085A26F04FA700CEBCECBDE1BA27037ED45F4FFE63
S123D460BCE4A7013986F120F6EC02FDBCE0FDBCE2BDDFF727037ED4C2A600850226037ED3
S123D480D4C285402716BDE03B27037ED4C2FEBCE2FFBCE0BDDFF727037ED4C2EC01FDBC2C
S123D4A098EC03FDBC9A86406F00084A26FACEBCECBDE1BA27037ED4C2BDDF8127037ED442
S123D4C0C24FFEBCE4A70139EC02FDBCE0EC04FDBC9CEE02EE008C2E002617FCBC10FDBC96
S123D4E098FCBC12FDBC9AFCBC9CC31000FDBC9E2027BDDFF72645FFBCE7A60085012604B8
S123D50086F42038EC01FDBC98EC03FDBC9AEC07830001F3BC9CFDBC9EFEBC98FFBC025F2E
S123D520CEBCECBDE1A627022012BDE0F9FEBC02BCBC9A270608FFBC0220E54FFEBCE4A7E3
S123D5400139EC02FDBCE0EC04FDBC9CEC06FDBC98EE02EE008C2E002615FCBC98F3BC109C
S123D560FDBC98FEBC98BCBC12232F86F52037BDDFF72632FFBCE7A6008501260486F420D9
S123D58025FCBC98E301FDBC98EC03FDBC9AFEBC98BCBC9A230486F5200CFCBC98FDBC025E
S123D5A0FEBC9CBDE1A6FEBCE4A70139EC02FDBCE0FDBCE2EC04FDBC9CEC06FDBC9EFEBCE4
S123D5C0E0BDD77025037ED675BDDFF7260586F47ED6758601B7BCE6FCBC9EB3BC9C8101AE
S123D5E023088302007CBCE620F4B6BCE6BDDEDE27037ED675BDDFC927037ED6753CFEBC33
S123D600E4A60884078AA038A700FCBC98ED01FCBC9AED03FCBC9EB3BC9CC3000124026CA9
S123D62006ED07FCBCE2FDBCE0C6093ABDE253C6073AC61FBDD67B4D270A81202706A700D1
S123D640085A26F04FA700CEBCECBDE1BA27037ED675FEBC98FFBC02BDE0D1CEBCECBDE106
S123D660BA27037ED675FEBC02BCBC9A270608FFBC0220E44FFEBCE4A701393CFEBCE0A6EB
S123D68000270608FFBCE038394F3839BDD67BBDD704241848484848B7BCE6BDD67BBDD788
S123D6A0042409BABCE6B7BCE64F0D390C39BDD67BBDD704243548484848B7BCE7BDD67B1F
S123D6C0BDD7042426BABCE7B7BCE7BDD67BBDD704241848484848B7BCE8BDD67BBDD704AA
S123D6E02409BABCE8B7BCE84F0D390C39A6002712812027030820F5A60027078120260301
S123D7000820F539271680302B1281092F0C84DF81112B0881162E0480070D390C39BDD62A
S123D7207BE6001126064D27030820F21B270581202701394F39A6002706BD7FE80820F6D0
S123D74039860DBD7FE8860A7E7FE886207E7FE844444444840F8B30813923028B077E7F09
S123D760E8A600BDD750A600087ED7548DF320F16D00272DA600272781202723811F2321C7
S123D780817E221D8122271981272715812A2711812F270D815C2709816027050820D50D95
S123D7A0390C39862DE600C54027028664BD7FE8862DE600C50127028672BD7FE8862DE6D5
S123D7C000C50227028677BD7FE8862DE600C50427028678BD7FE839FEBC94BCBC96222BA5
S123D7E0FFBC02CEBCECBDE1A627037ED164CEBCECA6002708FFBCE78D14FEBCE7C6403A62
S123D8008CBEEC26ECFEBC020820D07ED1E4BDD7A308BDD74BBDD76CBDD74BBDD76CBDD744
S123D8204BBDD76CBDD76CBDD74BBDD76C862DBD7FE8BDD761862DBD7FE8BDD761BDD74B43
S123D840BDD761863ABD7FE8BDD761863ABD7FE8BDD761BDD74BBDD736FEBCE7A600854068
S123D8602705862FBD7FE8BDD74139FEBCE0BDD6EDFFBCE0FFBCE2A60026022007EE008CD0
S123D8802F002618FEBC0CFFBC10FEBC0EFFBC12862FB7BC144FB7BC157ED1E4BDDFF727F1
S123D8A0037ED179FFBCE7A600854026037ED197850126037ED197EC01FDBC10EC03FDBC8A
S123D8C012CEBC14A60027030820F9FFBCE9FEBCE7C6103AFFBCE7FEBCE7A600271408FF23
S123D8E0BCE7FEBCE9A700088CBC932705FFBCE920E5FEBCE9862FA700086F007ED1E4FED8
S123D900BCE0BDD6EDFFBCE0FFBCE2A60026037ED185FEBCE2BDD77025037ED185BDDFF7DD
S123D92026037ED17FBDDFC927037ED18B8608BDDEDE27037ED18BBDDFC927037ED18B8689
S123D940C3A700FCBC98ED01FCBC9AED036F056F06CC1000ED07FCBCE2FDBCE0C6093ABD27
S123D960E253C6073AC61FBDD67B4D270A81202706A700085A26F04FA700CEBCECBDE1BA45
S123D98027037ED164CEBCEC6F00088CBEEB23F8FEBC9AFFBC02CEBCECBDE1BA27037ED111
S123D9A064FEBC0209FFBC02BCBC9822E927E77ED1E4FEBCE0BDD6EDFFBCE0FFBCE2A60029
S123D9C026037ED185FEBCE2BDD77025037ED185BDDFF726037ED17FFEBCE2BDD6EDFFBC49
S123D9E0E0A60026037ED185BDD6AE25037ED185FEBCE7FFBC9CFEBCE0BDD6EDFFBCE0A610
S123DA000026037ED185BDD6AE25037ED185FEBCE7FFBC9EBDDFC927037ED18B8601B7BC6B
S123DA20E6FCBC9EB3BC9C810123088302007CBCE620F4B6BCE6BDDEDE27037ED18BBDDFC6
S123DA40C927037ED18B86A3A700FCBC98ED01FCBC9AED03FCBC9EB3BC9CC3000124026CEE
S123DA6006ED07FCBCE2FDBCE0C6093ABDE253C6073AC61FBDD67B4D270A81202706A7008D
S123DA80085A26F04FA700CEBCECBDE1BA27037ED164CED091BDD736CEBC9CBDD76C862D97
S123DAA0BD7FE8CEBC9EBDD76CBDD741FEBC98FFBC02BDE0D1CEBCECBDE1BA27037ED16419
S123DAC0FEBC02BCBC9A270608FFBC0220E47ED1E4FEBCE0BDD6EDFFBCE0FFBCE2A600262D
S123DAE0037ED185BDD77025037ED185FEBCE2BDD6EDFFBCE0A60026037ED185BDD6AE258B
S123DB00037ED185FEBCE7FFBC9CFEBCE2FFBCE0BDDFF727037ED179A600850126037ED1D2
S123DB2097EC01FDBC98EC03FDBC9AEC07830001F3BC9CFDBC9ECED099BDD736CEBC9CBDCD
S123DB40D76C862DBD7FE8CEBC9EBDD76CBDD741FEBC98FFBC025FCEBCECBDE1A627037EDA
S123DB60D164BDE0F9FEBC02BCBC9A270608FFBC0220E47ED1E4FEBC10FFBC94FEBC12FFFB
S123DB80BC96FEBCE0BDD6EDFFBCE0FFBCE2BDDFF727037ED179FCBCE2FDBCE07EE121FEA7
S123DBA0BCE0BDD6EDFFBCE0FFBCE2A60026037ED185BDD77025037ED185BDDFF727037E2F
S123DBC0D179A600850226037ED19785402716BDE03B27037ED191FEBCE2FFBCE0BDDFF70D
S123DBE027037ED179EC01FDBC98EC03FDBC9A86406F00084A26FACEBCECBDE1BA27037E92
S123DC00D164BDDF8127037ED1647ED1E4FEBCE0BDD6EDFFBCE0FFBCE2A60026037ED185A9
S123DC20BDD77025037ED185FEBCE2BDD6EDA60026037ED185BDD77025037ED185FEBCE285
S123DC40BDD6EDFFBCE0BDDFF726037ED17FFEBCE2FFBCE0BDDFF727037ED179A600850232
S123DC6026037ED1973CFEBCE2BDD6EDFFBCE038C6103AC61FBDD67B4D270A81202706A770
S123DC8000085A26F04FA700CEBCECBDE1BA27037ED1647ED1E4FEBCE0BDD6EDFFBCE0FF80
S123DCA0BCE2A60026037ED185BDD77025037ED185BDDFF727037ED179FFBCE7FEBCE2BD9F
S123DCC0D6EDA60026037ED1855FA600271D84DF8152270B8157270B8158270B0820EBCA37
S123DCE00120F9CA0220F5CA0420F1FEBCE7A60084F8A700EA00E700CEBCECBDE1BA270313
S123DD007ED1647ED1E4FEBCE0BDD6EDFFBCE0FFBCE2A60026037ED185BDD77025037ED1A9
S123DD2085FEBCE2FFBCE0BDDFF727037ED179A600850226037ED197C6093ABDE253CEBCDD
S123DD40ECBDE1BA27037ED1647ED1E48647BBBFF8BBBFF9BBBFFABBBFFBBBBFFCBBBFFDE3
S123DD60BBBFFEB1BFFF27037ED1E4CEBCECBDE253CEBCECBDD76C862DBD7FE8BDD761862B
S123DD802DBD7FE8BDD761BDD74BBDD761863ABD7FE8BDD761863ABD7FE8BDD761BDD741DE
S123DDA07ED1E4FEBCE0BDD6EDFFBCE0A60026037EDE98BDD6AE25037EDE98FEBCE7FFBCFB
S123DDC0ECFEBCE0BDD6EDFFBCE0A60026037EDE98BDD68C25037EDE98B6BCE6B7BCEEFEE9
S123DDE0BCE0BDD6EDFFBCE0A60026037EDE98BDD68C25037EDE98B6BCE6B7BCEFFEBCE016
S123DE00BDD6EDFFBCE0A60026037EDE98BDD68C25037EDE98B6BCE6B7BCF0FEBCE0BDD6FD
S123DE20EDFFBCE0A60026037EDE98BDD68C25037EDE98B6BCE6B7BCF1FEBCE0BDD6EDFF83
S123DE40BCE0A60026037EDE98BDD68C25037EDE98B6BCE6B7BCF2CEBCECBDE2D5A601B71F
S123DE60BFF9A602B7BFFAA603B7BFFBA604B7BFFCA605B7BFFDA606B7BFFE8647BBBFF81B
S123DE80BBBFF9BBBFFABBBFFBBBBFFCBBBFFDBBBFFEB7BFFF7EDD4CCED0C7BDD7367ED123
S123DEA0E4BDD12BB7BCEB7EC000CED0BBBDD7365FCED243FFBCE7FEBCE76D00271AEE00E1
S123DEC0BDD74BBDD7365CC5032603BDD741FEBCE70808FFBCE720DFBDD7417ED1E4B7BCA6
S123DEE0E6FEBC04FFBC98FEBC08FFBC02CEBCECBDE1A6270139CEBCECA6002711FCBC98E9
S123DF00C30001FDBC98088CBEEC273520EBFCBC98FDBC9AA6002611FCBC9AC30001FDBCF4
S123DF209A088CBEEC270220EBFCBC9AB3BC984D2621F1BCE6221C271AFCBC9AFDBC98200F
S123DF40B8FEBC0208BCBC0A2206FFBC027EDEED86F239FCBC9A830001FDBC9A09FCBC9A5C
S123DF60FDBC986C007ABCE6270C09FCBC98830001FDBC9820EDCEBCECBDE1BA2701394FD8
S123DF8039FCBC98FEBC08810123068302000820F6FDBCE7FFBC02CEBCECBDE1A62701396C
S123DFA0FCBCE7C3BCEC18FCBC9AB3BC986F005D2709088CBEEB220E5A20F2CEBCECBDE1F9
S123DFC0BA2701394F3986F239FEBC94BCBC962223FFBC02CEBCECBDE1A6270139CEBCECFA
S123DFE0A60026024F39C6403A8CBEAC23F2FEBC020820D886F839FEBCE0FFBCE7FEBC947F
S123E000BCBC962233FFBC02CEBCECBDE1A6270139CEBCECA60027123CC6103AFCBCE7FD84
S123E020BCE0BDD71E3826024F39C6403A8CBEAC23E2FEBC020820C886F939EC01FDBCE77A
S123E040EC03FDBC02CEBCECBDE1A6270139CEBCEC6D002616088CBEEB23F6FEBC0209FFBE
S123E060BC02BCBCE722DE27DC4F3986F5397FBC007FBC017FBC027FBC03CEBCECBDE1A694
S123E080264CFEBCEC8C4D432644FEBCEE8C4653263CB6BCF081022635FEBCF1FFBC04FE07
S123E0A0BCF3FFBC06FEBD1BFFBC0CFFBC10FEBD1DFFBC0EFFBC12FEBD17FFBC08FEBD19AD
S123E0C0FFBC0A862FB7BC144FB7BC154F3986F139CEBCECFFBCE7FEBC9CA60008FFBC9CB9
S123E0E0FEBCE7A70008FFBCE78CBEEC270AFEBC9CBCBC9E220220DF39CEBCEC3A5FFFBC31
S123E100E7FEBCE7A60008FFBCE7FEBC9CA700BCBC9E270C08FFBC9CFEBCE78CBEEC26E1A0
S123E12039A60084A581A527037ED197EC01FDBC98FDBC02EC03FDBC9AEC07830001FDBC32
S123E1409ECEBCECBDE1A627037ED164CEBCECEC00814727037ED19D5D27037ED19DEC02E5
S123E160FDBC9CEC04FDBCE9FCBC9EF3BC9C830002FDBC9EC606CEBCECBDE1A627037ED138
S123E18064BDE0F9FEBC02BCBC9A270608FFBC0220E4BDD12BB7BCEBFCBCE0FEBCE93CFE31
S123E1A0BCE0FCBCE039BDE1E9BDE2028601B79FD28620B79FD77EE21F39BDE1E9BDE20264
S123E1C08601B79FD28630B79FD77EE239398604B79FD7BDE1E986E0B79FD68601B79FD159
S123E1E086EFB79FD7BDE1E939B69FD78480810026F739B69FD7840181002704B69FD139F6
S123E2004F39B6BC03B79FD3B6BC02B79FD4B6BC01B79FD5B6BC00840F8AE0B79FD639BD07
S123E220E1E9B69FD784088108260CB69FD0A70008BDE1F327E9394F39BDE1E9B69FD78430
S123E240088108260CA600B79FD008BDE1F327E9394F393637BDE25E5D26FA3332395F3CA1
S123E260CE9FC0BDE2C738A10627015CA7063CCE9FC2BDE2C738847FA10527015CA7053CD9
S123E280CE9FC4BDE2C738843FA10427015CA7043CCE9FC6BDE2C738843FA10327015CA775
S123E2A0033CCE9FC8BDE2C738841FA10227015CA7023CCE9FCABDE2C738A10127015CA7F7
S123E2C001B6BFF8A7003937A60148484848E600C40F1B33398607B79FCF4FB79FCDA600E4
S123E2E0B7BFF8A6013CCE9FCABDE32538A6023CCE9FC8BDE32538A6033CCE9FC6BDE325A2
S123E30038A6043CCE9FC4BDE32538A6053CCE9FC2BDE32538A6063CCE9FC0BDE325388602
S123E32004B79FCF39371644444444A701C40FE70033398647BBBFF8BBBFF9BBBFFABBBFAC
S123E340FBBBBFFCBBBFFDBBBFFEB1BFFF2621CEBFF8BDE2538647BBBFF8BBBFF9BBBFFA06
S11AE360BBBFFBBBBFFCBBBFFDBBBFFEB7BFFF39CED0A2BDD73639D7
S9030000FC
